:030000000219FDE5
:03000B000200AA46
:03002B0002018748
:03005B0002034459
:0300730002033154
:1000800002030406080C10182030406080040608A3
:100090000C10182030406080A0C00003070F1F0D17
:1000A0000D04050D050305030302C2AF306308C24A
:1000B0006385798AD2AF32C0D0C0E0206221E525C5
:1000C0006016E473E525F4C3334009758A00D263F2
:1000D000F57901D6F58AD262D0E0D0D0D2AF32C362
:1000E000E526334009758A00D263F57901F0F58A77
:1000F000C262E526F4602F30682520720DD0E0D072
:10010000D0C292C296C294D2AF32C292C296C29468
:10011000206F0C206609740ED5E0FDE57B4290D07F
:10012000E0D0D0D2AF32758A00D263757900C28D2B
:10013000D262211F01C4306805206602D29201C438
:10014000306805206602D29401C43068052066023A
:10015000D29601C4C29330680A2066077410D5E0B5
:10016000FDD29201C4C29530680A2066077410D58A
:10017000E0FDD29401C4C29730680A20660774106B
:10018000D5E0FDD29601C4C2AFC2AD53E6EFC0D0F8
:10019000C0E0D2D3D2AFE57A6009E5776005757724
:1001A0000041DE757701C2CEE52A6007207449154B
:1001B0002A21F87800790020742EE580307E01F441
:1001C00030E50278FF53DACF207E0343DA20307E19
:1001D0000343DA10C2D8C271E580307E01F430E505
:1001E0000279FFC3E89970CB306103752A18207437
:1001F00003752A18885CD27020740DE52B600415F5
:100200002B410843DA01C2D82070024177A85C2054
:100210006102C2702074367982B70431C3E894F069
:10022000400374F0F8E8C4540F28F87984B7030247
:10023000414DC313C3138721200802C313200A06AC
:10024000C3C898F8414D28F8500374FFF88822E598
:100250002D54066022206B1FE536C333C333F8E507
:1002600064C313C313F9C3952240028922E82522EF
:10027000F52250037522FF7882B60459852224A8FE
:1002800024C3E52495614002A861C3E89563400258
:10029000A8638825E566700241C8C3E8AA669A503B
:1002A00003E8FAE4F9EAC333FBE568F45B29400D9F
:1002B0002567F8E56760021567400B41C80AC3E58A
:1002C000679A5002056778FF8826C26FC3E52694B7
:1002D000F84002D26FC3E52594404002D26420CF9B
:1002E0000AD0E0D0D043E610D2AD32C2CF053AE515
:1002F0007A6009E57860057578006127757801787E
:1003000001E52A6005307402152AC3E55C940140BA
:1003100005755F006127756000756900E55F240160
:10032000F55F5003755FFFD0E0D0D043E610D2AD4B
:1003300032C2AF53E67F7592FA7593FFC260759132
:1003400004D2AF32C2AF53E6EFC2ADC0D0C0E0C0FE
:10035000F0D2D3D2AFA8FBA9FCE57A6007C3E913BA
:10036000F9E813F8C2D830710261B653DACF207EB3
:100370000343DA10307E0343DA20D271E580307E09
:1003800001F420E502618D88278928A1E353DACFA3
:10039000207E0343DA20307E0343DA10C2D8C271D4
:1003A000307402A1CF7800E580307E01F430E502A0
:1003B000A1CF885CA1B753DACF207E0343DA203087
:1003C0007E0343DA10C271206102818F53DACF209D
:1003D0007E0343DA10307E0343DA20C2D8D271881C
:1003E000578958C3E89555F8E99556F97B007E087A
:1003F0007A00C3E8948CE994005005755B00818114
:10040000882178A2E6A8216055C3E894C8E9940041
:100410005008E4D2E4FB7A0A815CC3E89468E9946A
:10042000015008E4D2E3FB7A0F815CC3E894D0E981
:1004300094025008E4D2E2FB7A1E815CC3E894A0E7
:10044000E994055008E4D2E1FB7A3C815CC3E8946E
:1004500098E994085008E4D2E0FB7A787E00C3E87B
:100460009559FCE9955AFD30E70AECF42401FCEDBE
:0E047000F43400FD755B00C3EC9AED9E500362
:10047E00755B018859895A8557558558567802A15A
:10048E00B7C3E89527F8E99528F9307C02A19B308F
:10049E007B02A19B307A02A19420750281B2E9FD04
:1004AE00E8FC81D1E9C313F9E813F8307902A1947D
:1004BE00E9C313F9E813F8307802A194E9C313FDE8
:1004CE00E813FC20612CC3EC941CED9402400281D5
:1004DE00E8ED701EC3EC94C850180529E52970028A
:1004EE001529C3E529940A5002A1CF755C00D2707C
:1004FE00A1CFE529600215297888E6F97400207FDE
:10050E00087896B90302789EE624FAFEE43400FFDA
:10051E00C3EC9EFCED9FFD9208B90310A208500794
:10052E00207609D276A13A307602C276A20850160B
:10053E00B9030DECF42401FCEDF43400FD02055476
:10054E0078007900A19BB90315EC33FCED33FDC3A4
:10055E00EC940AFCED9400FD50047C007D00C3EC8D
:10056E0094FFED9400400678FF7900A19BEC857214
:10057E00F0A4C5F0A2F733F8790040030205B7786E
:10058E00FF79000205B7E9C313F9E813F8307C0EC2
:10059E00E9600278FFC3E81338F8E43400F9C3E8E1
:1005AE0094FFE99400400278FF885CD270206102CB
:1005BE00A1CF741FF4552F4BF52FC274EB7002D2DE
:1005CE0074752A18307403752A0A306102A1E3206B
:1005DE00740353DAFE207403752B06D0F0D0E0D0EE
:1005EE00D0D2AD43E610327901020613790302062A
:1005FE0013790A020613791E020613796402061392
:10060E0079C80206137817E4D5E0FDD8FAD9F62298
:10061E007A147B7802063A7A107B8C02063A7A0DAF
:10062E007BB402063A7A0B7BC802063A7902E4C220
:10063E0095D5E0FDD294D5E0FDC294D5E0FDD295DE
:10064E00D5E0FDE920E002D29230E002D296E573C9
:10065E00D5E0FDE920E002C29230E002C296749627
:10066E00D5E0FDD9C9EAF8D5E0FDD8FBDBBEC295D1
:10067E0022C37C007D0075F00005F0EA33FAEB33FF
:10068E00FB50F6EB13FBEA13FAC3E9FFE8FEE89A18
:10069E00F8E99BF95004EFF9EEF8B3EC33FCED33C7
:1006AE00FDD5F0DFEDF9ECF822E889F08A20D2D4FE
:1006BE00F8A9F07B0030F70B7BFFF42401F8E9F486
:1006CE003400F9E88520F0A4ADF0F8E98520F0A417
:1006DE00AFF0FEED2EF974003FFA7C04C3EA13FA74
:1006EE00E913F9E813F8DCF48BF030F70AE8F42498
:1006FE0001F8E9F43400F9E889F0C2D4F8A9F0223F
:10070E007882B60403020769C3E55C9401400302D4
:10071E000733852224E4F544F545F546F547F548BB
:10072E00C26E0207697882E6FCD26EE522F5237866
:10073E003879C7AA40AB41C3EB13FBEA13FAEC14AA
:10074E006013C3EB13FBEA13FAEC14146007C3EB4C
:10075E0013FBEA13FAD17F8844894522C3E54495F9
:10076E0023F8E5459400F9500CC3E89480E994FF12
:10077E00401602079AC3E8947FE9940050030207DB
:10078E009A787F790002079A788079FF8849894A9A
:10079E0022E5492546F8E54A3547F9854A20E430F1
:1007AE000701F43548FA30E709C3EA94F040150220
:1007BE0007D8C3EA940F50030207D878FF79FF7A5F
:1007CE000F0207D8780079007AF0C3E524956150BE
:1007DE000AC374019524500B0207F6E54A20E70E72
:1007EE000207F6E54A30E706884689478A482278A6
:1007FE00A5E6FAC3E54933F8E54A33F91206B7E937
:10080E0030E70BC3E89480E994FF40130131C3E84D
:10081E00947FE9940050020131787F79000131789C
:10082E008079FFE820E715C3E52398F84009C3E86F
:10083E00940140030208587801020858E8F4240194
:10084E002523F8400302085878FF884B2278A6E645
:10085E00FAA847A9481206B7E930E70CC3E8940195
:0F086E00E994FF401602088DC3E894FFE9940057
:10087D00500302088D78FF790002088D780179FF09
:10088D00E920E715C3E54B98F84009C3E89401400A
:10089D00030208B478010208B4E8F42401254BF8EA
:1008AD0040030208B478FF88242278FFC2642069CF
:1008BD003D206A12D264C3E541940A4009C3E5257F
:1008CD0094405002C26479A1E76023E541601F7432
:1008DD00FF8541F0848539F0306A0375F005A4F881
:1008ED00C5F0600278FFC3E895645002A864886380
:1008FD0022C3E54094C8E5419400E56350031421FB
:10090D000F046002F563220209172275E890227820
:10091D0083E6FFE5E820ECF7A8BDA9BE0570C3E5A9
:10092D007094084052757000E9FA79A0E76044EAC6
:10093D007007E571601B020952C3E895716010E5FF
:10094D00715006600C1402095E0460F902095EE53F
:10095D0071F571C39472401B7561C0C3940440134B
:10096D00756180C39404400B756140C394044003CA
:10097D0075610075BB0822E5612410500274FFF506
:10098D00617982B7040221ABC3A861E524985002B6
:10099D00A824C3E895634002A86388258826E570DE
:1009AD00B4070375BB1022743279A787F0A4C5F084
:1009BD00A2F733F8C3E895614002A8618822882424
:1009CD00882588268864227540007541F022C2AFC3
:1009DD0075C820A8CCA9CDAA3A30CF010A75C82474
:1009ED00D2AFC3EA13FAE913F9E813F8AB3BAC3C09
:1009FD00883B893CC3E89BF8E99C20690A547FF940
:100A0D0030670241F54152AD3D8A3DF9EA9D547F73
:100A1D00FA600478FF79FFAE3EAF3F8B3E8C3FA866
:100A2D003BA93CC3E89EF8E99FF9C3E54113FBE5FB
:100A3D004013FAE82AF540E93BF54150067540FFB1
:100A4D007541FF419CAA40AB41AC40AD417E047F56
:100A5D0002C3EB940440021E1FC3EB940840021E18
:100A6D001FC3ED13FDEC13FCDEF7C3EA9CFAEB9DFF
:100A7D00FBEF6009C3E913F9E813F8DFF7EA28FA89
:100A8D00EB39FB8A408B4150067BFF8B408B41C37A
:100A9D00EB94025002D2673069047F0341C778920C
:100AAD00E6FFC3E537948240110FC3E53794A040AC
:100ABD00010FC3EF940640027F057E02E541C45449
:100ACD000FF9E541C454F0F8E540C4540F28F8C3BC
:100ADD00E89EFAE99400FB4009C3EA9402EB940006
:100AED0050047A02E4FB6141AA40AB41EBC4FEEA3B
:100AFD00C4540F4EFCC3EA9CFAEB9400FBC3E813FD
:100B0D00C313F8EA28FAEB3400FB8A408B41C3EBA0
:100B1D0094024002C2677802EBC4FE7B00EAC45423
:100B2D000F4EFAC3EA98FA4005C3940250027A02B6
:100B3D007892E6FF3060026141855192855293D2E1
:100B4D006043E680C3E49AF8E49BF9C3E833F8E91F
:100B5D0033F930670261D4E8FAE9FBD3E913FDE814
:100B6D0013FC88518952C3EF94036038EF20E00DD8
:100B7D00E82CF8E93DF9ECFAEDFB020B9DE828F8BD
:100B8D00E939F9C3E82402F8E93400F97AFE7BFF6C
:100B9D00C3EF9403400E8A538B54884D894E8C4F6E
:100BAD008D508108885389548A4D8B4E8C4F8D50B2
:100BBD003069127553F07554FF754FF07550FF7510
:100BCD0051F07552FF8108E8FAD3E813FC8851C340
:100BDD00EF94036020EF20E007E82CF8ECFA61F4C5
:100BED00E8282402F87AFEC3EF940340088A53885C
:100BFD004D8C4F810888538A4D8C4FE568C3335017
:100C0D0002646BF5683060028112753402D2604364
:100C1D00E680E52D5406602DA840A941C3E913F9DE
:100C2D00E813F8306904E92440F9C2AF53E67F7543
:100C3D009100C3E498F594E499F595759104D2600B
:100C4D0043E680D2AF22D265754300752000306C2B
:100C5D0003752040020C72D265754300752040303B
:0E0C6D006C0375200078017901206720E52DC9
:100C7B0054066002C2657914E541C313700104F890
:100C8B00C3941440027814306904781B791BC3E8B1
:100C9B0033F8C3E933F9206010E543600C30690386
:100CAB00D53404D26DA12A911A0543E59BF4544027
:100CBB00B52002A11430690908C3E89940011881D5
:100CCB00A120650A08C3E8994002817281A1C2651F
:100CDB00C2AF53E67F75910030671275940075951E
:100CEB00FC759104D26043E680D2AF8172AE40AF07
:100CFB0041C3EE33FEEF33FF50047EFF7FFFC3E4AF
:100D0B009EF594E49FF59581ECC3E5339401500275
:100D1B0081723065028172D802A12881A1C26DC295
:100D2B00AF53E67F75910085539485549575910467
:100D3B00854D92854E93D26043E680D2AFE52D541C
:100D4B00066008206A020533020D66306D0D206CBB
:100D5B000A2065071581158102161522780030646B
:100D6B00053065027801E53775F007A4F9E5F02841
:100D7B00F5F0E9A2F013A2F113A2F213F537C39425
:100D8B00785003753778C3E53795384008D266C27B
:100D9B0092C296C294306002A1A0854F9285509367
:100DAB00D26043E68022207D16C2AF754202C29507
:100DBB00D293306202D296D2AF759F40020FA0C27F
:100DCB00AF754202C295D297306202D292D2AF7502
:100DDB009F40020FA0307243207D20C2AF754203AB
:100DEB00900165757B20C296C297306204D294A1A4
:100DFB00FED295D2AF759F41020FA0C2AF754203D1
:100E0B00900165757B20C292C293306204D294C16B
:100E1B001ED295D2AF759F43020FA0207D17C2AF94
:100E2B00754203900140C296306202D294D2AF75E4
:100E3B009F41020FA0C2AF754203900140C2923096
:100E4B006202D294D2AF759F43020FA0207D16C2CF
:100E5B00AF754204C293D297306202D294D2AF756F
:100E6B009F43020FA0C2AF754204C297D293306268
:100E7B0002D294D2AF759F41020FA0307243207DF6
:100E8B0020C2AF754205900154757B08C294C29580
:100E9B00306204D292C1A4D293D2AF759F40020F9D
:100EAB00A0C2AF754205900176757B80C294C29546
:100EBB00306204D296C1C4D297D2AF759F40020F55
:100ECB00A0207D17C2AF754205900136C2943062E7
:100EDB0002D292D2AF759F40020FA0C2AF754205EE
:100EEB0090014AC2943062EBD296D2AF759F40020A
:100EFB000FA0207D16C2AF754206C297D295306205
:100F0B0002D292D2AF759F41020FA0C2AF754206BB
:100F1B00C293D295306202D296D2AF759F43020F25
:100F2B00A0307243207D20C2AF75420190017675CF
:100F3B007B80C292C293306204D296E14AD297D29E
:100F4B00AF759F43020FA0C2AF754201900154755C
:100F5B007B08C296C297306204D292E16AD293D2D6
:100F6B00AF759F41020FA0207D17C2AF7542019054
:100F7B00014AC292306202D296D2AF759F43020FE2
:100F8B00A0C2AF754201900136C296306202D29276
:100F9B00D2AF759F41C26622900134757B00C2921D
:100FAB00C296C294C293C297C295C26222788076CF
:100FBB00090876090876040876FF0876030876FF99
:100FCB0008760A087603087601087601788C760194
:100FDB000876FF0876FF0876FF0876FF0876FF088D
:100FEB0076030876FF0876FF0876FF0876250876E5
:100FFB00D00876280876500876040876FF08760223
:10100B0008760008767A0876FF08760108760108DC
:10101B007600087603087600227887E6FFC272BF57
:10102B000302D2727888E6C394036008C27DE6306F
:10103B00E102D27DC27E7889E630E102D27EC3EF37
:10104B0094026008758E01D27302105C758E00C21B
:10105B0073227880E6149000809378A5F67881E669
:0F106B00149000809378A6F67886E61490008D96
:10107A009378A7F67886E6F539C394025003753952
:10108A0002789CE67538FFB402037538A0B40303EE
:10109A0075388278A3E61490009A93F566120FA326
:1010AA0022227896E6FA7897E6FB7888E6B4030572
:1010BA00C3EB940EFB307F047A007BFFC3EB9AFCF0
:1010CA00C3948250027C827572000572EC8572F0BC
:1010DA00A4C3E5F0947D40F222D27F11AC1206043B
:1010EA007A007B007C101205FAE55C2AFA74003B50
:1010FA00FBDCF37C04C3EB13FBEA13FADCF7FEC256
:10110A007F11AC22E5EF20E6037520000520903F11
:10111A00FFE520146006901FFF146000930460032B
:10112A0075EF1253D9BF7581C043FF801205F5755B
:10113A00EF0243B203E5B3240220E70DF521E5E30C
:10114A0020E0068521B343E301120FA37580FF75E2
:10115A00A40075F13075D4DF75900375A5FC75F29E
:10116A00FC75D50175A60175E241C292C296C29478
:10117A00120609D293D297D2951205F5C293C29755
:10118A00C295120FA3E4F8F6D8FD756801120FB8DC
:10119A0012166E78988673753001C2AF12060E1257
:1011AA00061E12060412062512060412062C120640
:1011BA0004C2AF78FA79FA308507D9FBD8F7021C4E
:1011CA00001124115D11AB11AC78988673120FA32C
:1011DA0075A90075B680757A0075881075890275CB
:1011EA00C82475910475D84075A82275B80275E6A9
:1011FA0090759B80759D0075D10E75BCC075BB0836
:10120A0075BA1175E8801205F5D2AF120914753650
:10121A000053DACF207E0343DA20307E0343DA100C
:10122A0043DA01C2D8C27112060ED2617B037A0C6C
:10123A00E55B70077A0CDB030211BB12060420700F
:10124A00030211BBC270E55CC3940240E1E52F546E
:10125A001F855E5DF55EB55DD5DAD5C26153DACF1D
:10126A00207E0343DA20307E0343DA10C2D8C271EB
:10127A0078A2E67008D274E52F54E0F52FC275758E
:10128A002900120609307409C3E529940A4002D2DA
:10129A00751205FA78023074027800C3E55C98404A
:1012AA00F0C2AF12061E12061E12061ED2AF120698
:1012BA000E754C007888E6B40302619A1205FA7832
:1012CA008CE6C39401500302139AE530C39401508B
:1012DA000302139A207435C3E55C94FF500302138A
:1012EA009AC2AF120633D2AF120609C3E55C940163
:1012FA0050EFC2AF12061E1205FF12061ED2AF121F
:10130A000609C3E55C94FF40E90218167F02D27F02
:10131A0011AC120609C2AFC27F11ACAE5CC3E55C68
:10132A00947FD2AF40741205F5C2AF120633D2AF22
:10133A00DFDC11E3C3EE7897F612060E1216B0122E
:10134A0017997F0AD27F11AC120609C2AFC27F1168
:10135A00ACAE5CC3E55C947FD2AF50E61205F5C231
:10136A00AF12061E1205FF12061ED2AFDFD611E318
:10137A00EE24037896F612060E1216B01217C81249
:10138A00060911ACC3E55C94FF500241DE0218164F
:10139A00C3E55C954C4003855C4C120609780179DB
:1013AA0088E7B403027805C3E55C98400241BEC2EF
:1013BA00AF120633120633120633D2AF12060E7577
:1013CA003000E4F531F5320531E531F4703F05328C
:1013DA00789AE67819146012783214600D787D14C0
:1013EA00600878FA146003753200C3E53298401D2C
:1013FA00120FA31205F5153275310078998673C25A
:10140A00AF120633D2AF789886731206091205FF17
:10141A00E52A700530740221BB780120740278062F
:10142A00C3E55C9840A17888E6C39403600312067A
:10143A0009E52A70030211BBC2AF120FA3E4F52219
:10144A00F523F524F525F526F567D2AF7885E6C3A9
:10145A0033F565E4F544F545F546F547F548F57085
:0F146A00F52CF52DF53775700875BB101205F5CB
:10147900120918E5E820ECFBA8BDA9BEE97001F83E
:10148900887112091C75700875BB101124C2AF75DB
:1014990061FF1209B4852261852262852263D2AF78
:1014A9007522017524017525017526018560697507
:1014B9006A0175B69075A903757A017888E6B4034F
:1014C90007C27D307602D27DD268D26975330012A7
:1014D9000EFD120F2C1209D41209DB1209D41209BC
:1014E900DB1209D4120C6412070E120D67120DB12A
:1014F9001209DB120C53306E0312076A20670312BC
:1015090008B73067031208FE120D67120DE01209C1
:10151900DB120C64306E0312079F120D67120E570F
:101529001209DB120C53306E031207FD120D6712FC
:101539000E861209DB120C64306E0312085B120D61
:1015490067120EFD1209DB120918120C53120D67EE
:10155900120F2C12091C1209DB306932856461856E
:101569006462856069756A0179187A0CC3E53399F3
:10157900400FC269D26A8A35856461856463021540
:1015890097C3E55C940140030214ED02161D306A0D
:101599001D206C1AE535147006C26AD26B81EDF50F
:1015A90035C3E55C940140030214ED02161D75363E
:1015B9000078FA79A4E760027803C3E55F9850548C
:1015C900307404E52A604D7888E6B40317207D0558
:1015D900207607A1ED307602A1ED206C07D26C854B
:1015E9006461A12C78F0306C058564617820C3E5CD
:1015F9004198500281ED306C1BC26CC27D3076027D
:10160900D27DD26A75351285646181ED0536E55C56
:101619006002C120753600C2AF120FA37887E6FEBB
:10162900760211247887EEF6E4F522F523F524F500
:1016390025F526F565752C00752D0075A90075B67B
:1016490080757A00D2AF120609120FA378A4E6605A
:1016590006D293D295D297307409C3E536940440E3
:101669000221BB61CC901A0D78201216F2E520B444
:10167900550CA31216F2E520B4AA03021690120F14
:10168900B81216B00216AF901A0378807B0A1216A8
:10169900F2A308DBF9901A0F788C7B191216F2A3C2
:1016A90008DBF9901A2822C2AF12173112170B90D2
:1016B9001A00740E1216F7A374061216F7A37415FE
:1016C9001216F7901A0378807B0A1216F6A308DB24
:1016D900F9901A0F788C7B191216F6A308DBF91208
:1016E9001744121722901A2822E493F622E6438F10
:1016F90001538FFD75EF0275B7A575B7F1F0538FDB
:10170900FE22438F02438F0175EF0275B7A575B7A6
:10171900F1901A0DF0538FFC22901A0D7455D1F7E0
:10172900901A0E74AAD1F7227A3079D07820901ABB
:1017390040D1F2E520F709A3DAF7227A3079D0907F
:101749001A40E7D1F709A3DAF922AB74A875BB01EE
:10175900027980BB02027981BB03027982BB040250
:101769007984BB05027986BB06027992BB070279A7
:1017790087BB080279A3BB0902799CBB0A02798855
:10178900BB0B027989E8F7227C0512060EDCFB22E5
:10179900C2AF12061E12062512062C1206331205B6
:1017A900FF12061E12062512062C1206331205FF19
:1017B90012061E12062512062C120633D2AF22C2B9
:1017C900AF12063312062C12062512061E1205FF49
:1017D90012063312062C12062512061E1205FF12D6
:1017E900063312062C12062512061ED2AF22AE743B
:1017F900AF75C2AF12061E12061E12061E1205FF93
:10180900DEF21206331205FFDFF8D2AF2212179962
:101819001217911217917574017575017576001279
:1018290017F77C05AD5C12060EC3ED955C70F5C328
:10183900E55C9401400AC3E55C94FF403702185AFD
:101849001217531216B0121799C2AF75EF12121769
:1018590091DCD10576C3E5769403500280C1121755
:0F186900910575E5741490009F93F808C3E57519
:1018780098500280A81217911217910574C3E57445
:10188800940C50028094120FB81216B0C2AF75EFC4
:041898001212179180
:0319FD0002110EC6
:101A00000E0615090904FF03FF0A03010155AA0187
:101A1000FFFFFFFFFF03FFFFFF25D0285004FF0259
:091A2000007AFF0101000300FF40
:101A400023475F556C74726132304123202020207F
:101A500023424C48454C492346333930232020202B
:101A60002020202020202020202020202020202076
:101C0000C2AFC2D353D9BF7581C043B20343FF8073
:101C1000752438752503B1C975EF0275E24043F1AB
:101C20002053A4DF75D4FFD2857DFA780379E67C52
:101C300010752200752300901DD67B0675249875BB
:101C400025013085028142208508D8FBD9F9DCF7CF
:101C500081B4308508D8FBD9F9DCF781B4B189E4C7
:101C600093A3C39A6004DDC381B4DBDBB17B600264
:101C7000812B7B08E493FAA3B15CDBF87A30B15C8A
:101C8000752200752300B17BEAFCEBFDC3ED94FEE9
:101C9000400EB17B8A278B28ED30E0048A828B834B
:101CA000B17B7AC270D8C3ED94FE601350CEBD00F4
:101CB00025EC60097520007521FF0200008100A855
:101CC00027A9280809D804D90281D3B17FEA89AAB3
:101CD000F281C50D81A0C3ED94035049EDA2E092BD
:101CE000007AC5C3E5829400E583941C50902000DF
:101CF00010438F02438F0175B7A575B7F1F030001F
:101D00001FA827A9280809438F01538FFDD804D99C
:101D100002A12089AAE275B7A575B7F1F0A3A10DBC
:101D2000538FFC817C7AC1BD030CE493A3FAB140CC
:101D3000DCF8B138817C817EAA22AB23B15CEBFA5E
:101D4000EA6222752608C3E52313F523E52213F57D
:101D50002250066323A0632201D526EAB1C9B1C986
:101D600075260AEAF4200102D285300102C285B14B
:101D7000C9C3134002C201D526EB22B17FEAFB2082
:101D80008502A17F308502A184752608AE24AF2587
:101D9000C3EF13FFEE13FEB1CDB1C9C3EA13308513
:101DA000024480FA30E703632201C3E52313F523DD
:101DB000E52213F52250066323A0632201D526D91C
:101DC000E52265236523F52222AE24AF250E0FDE22
:101DD000FEDFFCD20122424C48656C693437316326
:041DE000F390060175
:00000001FF
